:020000040000FA
:1000000000306500FF3066000515A001A201A301C4
:100010000A30A100A00A210820020318A0010A2822
:100020000800080090309D0029203C309D002920C8
:100030007F309D00292008000D309C00FF309B0080
:10004000FF309A009A0B22289B0B20289C0B1E281D
:100050000800051118309F009F0B2C2808309B00CA
:100060009D0C0318362800000511392805150000DD
:10007000000017309F009F0B3B289B0B302800008F
:10008000000000000000000005151A309F009F0BC3
:0400900047280800F5
:02400E00F23F7F
:00000001FF
